:02000000400AB4
:10008000D70C020066006800F90C0600010C27007E
:100090000000040C8801280026006606B30A500AF6
:1000A000040C880128002600E702480A570A040CBD
:1000B000880128002600020C880128002600040C74
:1000C000880128002600E80C270000000000040C2E
:1000D0008801280026000606A40A00000000040C7F
:1000E000880128002600E702660A760A060C8801C5
:1000F00028002600E80C2700490A0000040C8801AB
:10010000280026006606B30A850A040C8801280028
:100110002600E7027D0A00000000040C8801280088
:100120002600020C880128002600040C8801280003
:100130002600630C270000000000040C8801280042
:10014000260006076E0A00000000040C8801280043
:100150002600E7029C0AAC0A060C8801280026004B
:10016000630C27007E0A0000040C8801280026008A
:100170006606B30ABB0A040C88012800260006069E
:100180008C0AC20A040C880128002600C70A570AF4
:021FFE00E90FE9
:00000001FF
